:400000000010002011000000650F0000650F000010B500F0C7FFC04670B5194C23688022D20213432360182001F02EFA2268154B13402360144A154B1A603022144B1A603E
:40004000203A144B1A601032134B1A6082221206124B1A6000252560114A124B1A60124A124B1A60124A134B1A601349092001F0B1F9092001F098F9104B1D6070BDC04687
:4000800000010B40FFFFFBFF0600008004010B400C0202401C0202402002024008010B400E0000800000024017000080400002403801008080000240991600000C020B4052
:4000C00010B572B60122244B1A7000240FE023486200131959000B00411889881A5AC31858880004104300F01DFF0134E4B2012CEDD91A4801000C311C3000F0F9FE184A98
:40010000184B1A6099231B04174A1360174A1360174A13600122174B1A60174A117806230B43DBB213700822144B1A60C0221201134B1A600223134A1360134A1360134A29
:4001400013601349134A1160134A1360FFF764FF00F0FEFE10BDC0461C700F40084A000099EE00000C00014010500F4020500F4030500F402000004000700F400001044058
:4001800008010440000204401802044000030440B10D0000080304401803044010B5064C2378002B07D1054B002B02D0044800E000BF0123237010BD800100200000000089
:4001C00058470000084B10B5002B03D00749084800E000BF07480368002B00D110BD064B002BFBD09847F9E7000000008401002058470000C00000200000000010B562B681
:4002000000F0EAF900F012FA00F028FA00F02AFA00F02CFAF6E7C04610B5064B0020185E0B23054A054900F0DDFA02F007F8044B188010BDC2020020AC02002044030020D4
:40024000C4020020F0B585B0254B04255D5F254B00241C5FA54211DD234B01221A7000225A702C1B322C03DD204A214B1A8035E01B4B00229A5E1E4B1A802FE0184B062059
:40028000185E844211DD184B01225A7000221A70641B322C03DD154A154B1A801EE0104B02229A5E124B1A8018E00D4B00229F5E02269E5F02F042FD0390280002F03EFDE9
:4002C000051C200002F03AFD00963B00039A291C00F052FA01F0B2FF054B188005B0F0BD5C030020C20200209C010020FF7F0000C402002010B5054B0C229B5E002B02D0FC
:40030000FFF78AFF01E0FFF79DFF10BD5C03002070B5012000F046FF002845D0002000F055FF224B1880224B9B78592B10D85900204A885201331E4A937035E05E001D4A5C
:40034000B25E1400D517001969410133DBB202E0002300200021592BF0D95A22002301F01DFF01B2002000F047FF134C208001220F4B9A700D4B1A880E4B1A80FFF7BAFF7F
:400380000023E05E0D4C608002F0D8FC0C4902F0FFF80C4902F016FA01F050FFA0800023E15E094800F008FA70BDC046A80200209C010020F4010020C2020020C4020020AA
:4003C00000002C420000C8426447000010B50A304000044B1A88044BC25200F03FFA00F049FA10BDC20200205C030020F0B583B0644C1423E25E644B1A801621625E5A80A2
:400400001821625E9A801A21625EDA801C21625E1A811E21625E5A812021625E9A812221625EDA812421625E1A822621625E5A822821625E9A820023E05E544D288003F022
:40044000A1FA06000F000223E45E200002F076FC03F0DAFA4E4A4F4B0090019102F0E2FF02000B003000390002F0B0FC03F054FA6880474A484B0098019902F0D3FF02009A
:400480000B003000390002F0A1FC03F045FAA880424A434B0098019902F0C4FF02000B003000390002F092FC03F036FAE880384A3C4B0098019902F0B5FF02000B0030003F
:4004C000390002F083FC03F027FA28810022364B0098019902F0A6FF02000B003000390002F074FC03F018FA68812C4A2F4B0098019902F097FF02000B003000390002F051
:4005000065FC03F009FAA881294A2A4B0098019902F088FF02000B003000390002F056FC03F0FAF9E8811A4A234B0098019902F079FF02000B003000390002F047FC03F093
:40054000EBF928821D4A1E4B0098019902F06AFF02000B003000390002F038FC03F0DCF96882AC82082309E01A00083A52000549505E5900134A88520133DBB2272BF3D9E7
:4005800003B0F0BD5C03002044030020AC0200209A9999999999B93F9999C93F333333333333D33F9999D93F0000E03F3333E33F666666666666E63F9999E93FCDCCCCCC15
:4005C000CCCCEC3FC402002010B500F0D1FD00F0DFFDFFF70BFF10BD10B5FA20800000F031FF00F023FD0C4800F022FD00F058F90A4800F01DFD0A4800F01AFDFFF7E4FF75
:40060000084800F015FD00F0ABF8074800F010FD00F064F910BDC0466C470000804700008C470000A0470000B047000010B50A4B1B885A0605D540229343074A1380FFF735
:4006400067FE054B1B88DA0603D510229343024A138000F053FA10BDA201002010B500F0E3FB10BD10B500F05DF910BD7047C04610B500F093FE38490A8801231A4392B2A3
:400680000A8036490B88013B9BB20B80002B06D10721324B198040231A432F4B1A802F4A5388013B9BB25380002B07D114222B4B5A80294A118880230B431380274A938821
:4006C000013B9BB29380002B07D10A22234B9A80214A118802230B431380204AD388013B9BB2D380002B08D1FA2292001B4BDA80194A118810230B431380184A1389013B40
:400700009BB21381002B07D13222144B1A81124A118808230B431380104A5389013B9BB25381002B07D164220C4B5A810A4A118820230B431380094A9389013B9BB293811B
:40074000002B07D11922054B9A81034A118804230B43138010BDC046A2010020C400002010B500F0CBFD00F0FDFD024800F008FE10BDC04671060000F8B50D1C161C1C0053
:4007800002F034F9071C069B181B02F0D7FA391C02F018F8071C291C301C02F027F9011C381C01F0F5FE051C200002F0C7FA011C281C01F077FDF8BD10B58EB00C0000F080
:4007C00037FC2200054901A803F0A2FB01A800F02FFC034800F02CFC0EB010BDC04700007C470000F8B500254C5F844204DB0023D05E02F0A3FA2DE0174CA44663445B0043
:40080000CC5EA04206DBD05E02F098FA22E00133DBB200E001231E005D004C5FA042F6DC03D1505F02F08AFA14E00B4B9C4666447600895F431A555F905F2D1A5D43641AE6
:40084000001902F07BFA041C280002F077FA211C01F09EFEF8BDC046FFFFFF7F10B542220249034800F06CFF10BDC046C44700005C0300204023084AD15C084AD154002359
:4008800006E05A000449505E044950520133DBB21F2BF6D97047C046C44700005C03002010B500F04BFF012000F0CCFD4023064AD35C002B04D142220349044800F040FF07
:4008C000FFF7D8FF10BDC046C4470000C84B00000A22014B1A707047AD01002010B500F08DFFFFF7F5FF10BD30B5FF22FF2508E003785340084AD25C6A400849CD5C2100D6
:4009000001304B1EDCB20029F2D12802104380B2034B5D701A7030BD08480000084900006404002010B5194B1C78002C28D000F0F7FF012000F086FD2100154800F0E4FF8D
:40094000144B1B68DB06FBD5124B1B689B05FBD50F4C96220021200003F0D1FA8022520000210D4803F0CBFA00F06CFF96220021200003F0C4FA20220021084803F0BFFAFC
:40098000024B00225A801A809A8010BDAE010020C0030020800F074090040020A0030020002807D0062803D90F38C0B2012801D8012000E000207047F8B500F02FFF050002
:4009C000C4B200F02BFF002845D0474B5B78DBB2464A1278934209D0FF222A400021424803F08DFA00F02EFF002434E0052000F029FD00F013FF0400C3B2022B22D93A4B08
:400A00009878C0B2FFF7CCFF002809D1FF2222400021354803F073FA00F014FF00241AE00F2000F00FFD00F0F9FEC4B2072C12D8FF22024000212C4803F061FA00F002FFF3
:400A4000002408E0FF2202400021274803F057FA00F0F8FE0024072C40D9012000F0F2FC214A937892780F3B59424B41103A51424A41134318D01C4BDD790A35EDB2002488
:400A80000DE0012000F0DEFC00F0C8FE6B1E984203D9012000F0D6FC06E00134A4B2144B1B796B439C42ECDB124F20220021380003F025FA00F0B2FEC4B2FF2505400E4EE6
:400AC0002A003100380003F011FA701E2A00002103F015FA00F0B6FE012300E0002398B200022043F8BDC04690040020AD010020D4000020A00300209104002010B5FFF7AC
:400B00005BFF030ADBB2012B09D1074B00229A71FF321040A022D2001043588003E0E022D200014B5A8010BDAE01002070B506000D00094C96220021200003F0E0F9074BDF
:400B40001B7823706670A57003212000FFF7CCFEE070000A207170BDC0030020AD01002010B5034A034B1A80FFF7E0FF10BDC04605FCFFFFAE010020F0B5474680B4314A46
:400B800094782402D3781C4317793F0253791F437B1E9BB2092B04D902218420FFF7E0FF4DE0294B9C4204D902218420FFF7D8FF45E03D002600254B1B1B9F4204DD0221C4
:400BC0008420FFF7CDFF3AE0214B9C4204D802218420FFF7C5FF32E01E4B984696220021180003F08CF91C4B1B7842461370042353707F009770063CE3B203240CE0621C2F
:400C0000D2B258001549405E124907120F550234E4B288540133DBB2114AB218AA189342EDDB0C4D21002800FFF75EFE631CDBB22855000A0234E4B2E8540A4B1C8004BCD7
:400C40009046F0BDA00300200F2700001027000005270000C0030020AD010020C4020020FAD8FFFFAE01002010B501218120FFF777FF10BD10B501218220FFF771FF10BDE2
:400C800010B501218520FFF76BFF10BD10B501218F20FFF765FF10BD10B526498B781B02CA781343087900024A791043072B04D802218620FFF754FF3AE0122B04D90221C2
:400CC0008620FFF74DFF33E00F2B04D10A2818D8FFF77CFB15E0083B5B00174A9852FFF7BDFDFFF7C7FD082309E01A00083A52001149505E5900114A88520133DBB2272BA8
:400D0000F3D9FFF773FB002305E00A4AD15C0C4AD1540133DBB2052BF7D9094C06212000FFF7E2FDA071000AE0710822054B1A8010BDC046A00300205C030020C4020020D2
:400D4000C0030020AE01002010B502219020FFF707FF10BDF0B5474680B404000F003F2804D902218320FFF7FBFE3AE00D00060040231B1A994204DD02218320FFF7F0FEC3
:400D80002FE0194B984696220021180003F0B7F8164B1B7842461370032353707F009770E0B203240CE0631CDBB24100104A895E0D4A0F1217550234E4B2D1540130C0B236
:400DC000AB199842EFDB084D21002800FFF78CFD631CDBB22855000A0234E4B2E854054B1C8004BC9046F0BDC0030020AD010020C4020020AE01002010B50A4B9878000212
:400E0000DA781043197909025B7919434B1E9BB23F2B04D902218320FFF7A2FE01E0FFF799FF10BDA003002070B52D4B5B881A0A052A53D1DCB2A61EF1B22A4D2800FFF767
:400E400053FDC2B2000AC0B2A95D631EEB5C521A51424A41C31A5842434113423ED0214B1A78214B1B789A4234D11E4B5B78012B02D1FFF7F9FE31E0022B02D1FFF7FAFE77
:400E80002CE0032B02D1FFF7B7FF27E0042B02D1FFF772FE22E0052B02D1FFF7F1FE1DE0062B02D1FFF7F8FE18E00F2B02D1FFF7EDFE13E0102B02D1FFF746FF0EE00B49CF
:400EC000074A1180802040420343D8B20121FFF72DFE03E0C022D200014B1A8070BDC046AE010020A0030020AD01002005F9FFFFF0B50025002711E0BB00C658F3B2FF224E
:400F0000964308E06A008A181478A419527822700135013BDBB2002BF4D10137012FEBD9F0BDC04610B50A00002102F0E8FF10BD064B1B68002803D080221206134301E01B
:400F40005B005B08014A13607047C04680031A4010B50222024B1A600120FFF7E9FF10BD00031A4010B502F095FF03680C2B00D1FEE7FEE710B50300084A1068C318084A3B
:400F80009A1A802A02DC054A136005E002F082FF0C2303600120404210BDC046F00000209805002070B50F4E0F4D13E029686B68AC68002202E001C901C30432A242FAD146
:400FC000E868002202E0002102C304328242FAD11035013E002EE9D102F062FFFFF70EF9FEE7C04601000000B84B000010B500230AE0032B03D89A000949505800E00948A7
:401000009900094A885001332F2BF2D9FFF758F88022D205116801230B43136010BDC04600000000650F0000000000207047C04670B505000078012404E000F021FD285D14
:401040000134E4B20028F8D170BDC04610B503210E2000F0D1F924490E2000F0BBF90122224B1A60224B1B68002B01DA214900E02149224A13680B431360214A214B1A60C4
:40108000214A224B1A600023214A1360214A22490A6022490A6022490A688020400202430A60204A1360204A136001331F4A136002211F4A11601F4908681F4A02401343BA
:4010C0000B6000230DE09A001C4951188020C0000860580000241A4944521A481A4950500133002BEFD010BD5512000020001A4080031A40400210534002005300001A402E
:40110000AC00008004001A400000FF0718001A401C001A400200020010001A4014001A4000031A4028021A4038021A4018021A40000F1A4030001A40FFFFFFDF80001A40C9
:401140006C040020204E00006804002010B5074B1B68002B08DB054A1368802109060B4313600A2000F086F910BDC04600001A4010B5064B1B78002B04D1FFF767FF012214
:40118000024B1A70FFF7E2FF10BDC046B9010020034A1368802149020B4313607047C04604001A40020083070CD0074B1B680120184001D19307F8D4002804D00122024BEA
:4011C0001A6000E00020704710021A4010B5041E02D0002000F0FCF8002C07D1A400054B9C46644420680004000C00E0002000B210BDC04680011A4070B504000D000028BD
:4012000002D0002000F0E4F863000F4A995A09B2691A09B20D484843002906DDA3000C4A9A58D30F9A18531006E0A300084A9A58D30F9A18521053421818A400044BE158C6
:4012400000F0C0FE00B270BD6C0400201027000068040020014B1A681A60704710021A400004000C014B18607047C046080105400004000C014B18607047C0461401054059
:4012800070B504000D0000F071FCAC40024B1C6000F070FC70BDC0460800054010B500F065FC064A116801230B43136000F062FC18210120FFF7E4FF10BDC04600000540AD
:4012C000014B18607047C0463801054010B580229204074B1A600C22064B1A600120FFF7EFFF0548FFF7C4FF0020FFF7B9FF10BD0001054024010540E703000010B5064BD7
:401300001B78002B04D1FFF7E1FF0122024B1A70FFF7C4FF10BDC046BA0100207047C046014B18647047C0460000002010B5040000F01CFC044A1368C0218B43A4011C4334
:40134000146000F017FC10BD00E400E00122014B1A60704700E100E00122014B1A60704780E100E010B5FFF7F7FF0448FFF7D8FF0320FFF7DBFFFFF7E9FF10BD1D1300008B
:4013800010B50400FFF7E8FF2000FFF7C9FF0320FFF7CCFFFFF7DAFF10BDC0460122014B1A60704780E200E01F2318401E3B8340014A13607047C04600E100E01F231840B5
:4013C0001E3B8340014A13607047C04680E100E001BE704770B504000D001F2802D90020FFF7F6FF1034A40080239B059C4664442068256070BDC04670B504000E000329E4
:4014000002D90020FFF7E4FF1F2C02D90020FFF7DFFF03252540ED00063500F0A7FBA408A400074B9C46644421680323AB4099430B003100A9401943216000F09BFB70BD20
:4014400000E400E010B5040006E0084B586800F083FB074B9C46644480231B029C42F4D8024B9868604300F077FB10BD000100200080FFFF10B5034B1B7B584300F06CFBD9
:4014800010BDC04600010020F0B557464E46C0B483B0040000F06AFB0190E71E2D2F74D83F4B1B78DBB29C4208D83E4B1B78DBB29A463D4B1B78DBB2994631E03B4B1B7882
:4014C000DBB29C4208D83A4B1B78DBB29A46394B1B78DBB2994623E0374B1B78DBB29C4208D8364B1B78DBB29A46354B1B78DBB2994615E0334B1B78DBB29C4208D8324B68
:401500001B78DBB29A46314B1B78DBB2994607E02F4B1B78DBB29A462E4B1B78DBB299462D4BDE5D2F2E09D92A2C07D919222B4B1A60052000F010FB192503E0274B1D68CC
:401540003F231D40B54206D9234BDA5D234B1A60052000F001FB1F4B9C4664442378DBB21F4A13601F4B52461A601F4B4A461A600520FFF77FFFB5420AD2174BDA5D174BE9
:401580001A60052000F0E8FA02E00020FFF720FF019800F0EFFA03B00CBC91469A46F0BDC0F1FF0FC1F1FF0FC2F1FF0FC3F1FF0FC4F1FF0FC5F1FF0FC6F1FF0FC7F1FF0F3E
:4015C000C8F1FF0FC9F1FF0FCAF1FF0FCBF1FF0FCCF1FF0FCDF1FF0F2C4A00002CFF0B4028FF0B401CFF0B4020FF0B40034B1868C0231B02184000D00120704700010B40EA
:4016000010B500F0B3FA044A1368C02109020B43136000F0AFFA10BD00010B4010B500F0A5FA08490A68084B1A408024E40122430A600A6813408022120213430B6000F0D8
:4016400099FA10BD00010B40FF3FFFFF70B5050000F08CFA0400FFF7C9FF002803D0FFF7DDFF012100E0002108482840084A1568084B2B40184310601368012901D1FFF7B3
:40168000BFFF200000F076FA70BDC0460404040010020B40FBFBFBFF10B5244B1B685B0715D5234B1B685B070ED5224BD969042001401F4C22688A432260DA698243DA618C
:4016C0001B69002B00D098470420FFF7BFFF174B1B685B0518D5164B1B685B0510D5154BD9698022D2001140114802688A430260D969114A0A40DA615B69002B00D0984740
:401700008020C000FFF7A2FF084B1B685B030CD5074B1B685B0304D5064B9B69002B00D098478020C002FFF791FF10BD10020B4014010020BC010020FFFBFFFF7047C04689
:40174000F0B54F464646C0B4A1B0804617000E008A1880231B029A4229D8CC0BC909FF230B40994624024C44E4010020002519E0B44207D3BD4205D24246525D6946CA543C
:40178000013502E022786946CA540134013300E000237F2BECD96946484600F003FA01239C46E144BD4203D20028F1D000E00120012801D90120404221B00CBC90469946C8
:4017C000F0BDC04610B50B20FFF7EEFD10BDC04610B500F043F910BD10B500F0CDF810BD10B5054A1368802109060B431360FFF7E9FFFFF7EDFF10BD0000074010B5064BA3
:401800001B78002B04D1FFF7E7FF0122024B1A70FFF7E6FF10BDC046DC010020074B1B68074A1268934203D3054A1068181A04E0034A10681B1A581CFF3070478C04002068
:401840007404002010B50B20FFF7B8FD0B4B1A680B4B1A6000220B4B1A700B4B1A68802149020A431A601968084A0A401A60084A084B1A600B20FFF797FD10BD7404002030
:401880008C0400207004002004030740FFFFFEFFED0F0000C00F0740144B1A68144B1B689A4208D1134B1B680F221340082B02D0114B186019E00D4B1A6801320C2A00D1C6
:4018C00000220B4B1B689A42FBD002230B490B60C0B20B49885405490A600A4A1268134203D1084A11680B43136070477C040020780400200802074040020740800F0740E2
:4019000080040020880F074070B506000D00002403E0305DFFF7C0FF0134AC42F9D370BD10B50B20FFF74AFD0C4B1A680C4B1A600C4A136802218B4313600B4B1A68802103
:4019400049020A431A601968084A0A401A60084A084B1A600B20FFF727FD10BD780400207C040020880F074004020740FFFFFEFFF3070000800F074010B51F4A1F4B1A6049
:4019800000241F4B1C601F4A1F4B1A601F4B204A136007211F4A11601F4A146006391F4A11601F4A13601F4B1C600B20FFF706FD03210B20FFF720FD1B490B20FFF70AFDBD
:4019C0001A4B1C601A4B1C601A4B1C601A4B1C6004221A4B1A601A4B1C601A68194B1A80194B1C60194B1C60194B1C70194B1C60194B1C6010BDC04607000002000007406A
:401A00004000074001000A004800074007000080000307400403074010030740440007400002074004020740C91D0000880E0740C80E0740480F0740080F0740C80F0740F1
:401A4000880F0740E40100208C04002074040020700400207C0400207804002005490B68F0229343603A13430B60034B1A88034B1A6070470C000140E4010020880F0740C8
:401A8000FEB5494652465B460EB407462E4909688A462E4A12682E48022100F009FA03002A480068C0182A4900F002FA06001F3EB346234A126801219140C9430C000125DE
:401AC000002600F053F8814651460B6823400B605846043000F040F83800F040284090400B68234003430B60584600F035F80136072EF1D900200130012090400B682340BC
:401B000003430B605846063000F026F8484600F031F8C046C046C0460EBC894692469B46FEBDC046C046C046C046C046C046C046C046C046C046C046C046C046C046C046F2
:401B4000FC000020F8000020F40000201001002000C20100000000000230800804D0C0460138FDD1C046C046C0467047EFF3108072B6704780F310887047C046024B1A68DD
:401B8000024B1A600020704708010B40E8010020024B1A68024B1A6000207047E801002008010B40F0B5474680B4A6B00500002325932493FF2800D9EFE0002900D1ECE078
:401BC000802204A802F092F9022300200021002408E09A0002AE9259002A02D0891810431C000133212BF4D9002903D1002803D1002602E0002600E00126002E06D0A30045
:401C000002AA9F58002202A95A5000E00027664B02937F230393654B02AA1A606449654A1160C0461B681B0F1B07F0221206934204D15E4B1B68FF2213400DE05B4B1B6803
:401C40001B0F1B07A0221206934204D0574B1B68FF22134000E000232593259B002B00D09DE0FFF783FF0190FFF788FF2490259B002B25D1504A029202992A040A43029216
:401C80004A4A02A911604D484A490860C0461268120F1207F02109068A4204D1434B1B68FF2213400BE0414A1268120F1207A02109068A4203D03D4B1B68FF221340259314
:401CC000259B9846002B59D1002E57D08022002104A802F014F9A40002ABE750324B02937F230393314B02AA1A603149314A1160C0461B681B0F1B07F0221206934205D1AA
:401D00002A4B1B68FF221A4090460CE0274B1B681B0F1B07A0221206934204D0234B1B68FF221A40904643462593259B002B25D1234A0292029A2D04154302951B4A02A979
:401D4000116020481B490860C0461268120F1207F02109068A4204D1144B1B68FF2213400BE0124A1268120F1207A02109068A4203D00E4B1B68FF2213402593249B002B91
:401D800007D1FFF705FF2490249B002B01D0249B25930198FFF7EEFE01E004232593259826B004BC9046F0BDB6D70000080000400400008004000040B6D8000005000080AA
:401DC000B6D900000600008010B5284B1B68002B00D09847264B1B685B071FD5254B1B68013380225200934200D10023224A1268934205D1214B1B682022214B1A7006E06D
:401E00001E4A1268D2B21F49CA541A4A13601E4B1B681B07E2D104221C4B1A601C4B1B689B0721D51B4B1A681B4B1B689A4213D0194B1B6801330C2B00D10023174AD25C30
:401E4000D2B217490A60144A1360164B1B680F221340082BE6D104E0134A136802218B4313600222114B1A6010BDC046E0010020CC0F07408C04002074040020400307400F
:401E8000700400209004002008030740C00F07408C0F07407C04002078040020800400204002074008020740880F0740800F0740002243088B4274D303098B425FD3030A89
:401EC0008B4244D3030B8B4228D3030C8B420DD3FF22090212BA030C8B4202D31212090265D0030B8B4219D300E0090AC30B8B4201D3CB03C01A5241830B8B4201D38B033E
:401F0000C01A5241430B8B4201D34B03C01A5241030B8B4201D30B03C01A5241C30A8B4201D3CB02C01A5241830A8B4201D38B02C01A5241430A8B4201D34B02C01A5241E8
:401F4000030A8B4201D30B02C01A5241CDD2C3098B4201D3CB01C01A524183098B4201D38B01C01A524143098B4201D34B01C01A524103098B4201D30B01C01A5241C30837
:401F80008B4201D3CB00C01A524183088B4201D38B00C01A524143088B4201D34B00C01A5241411A00D20146524110467047FFE701B5002000F0F0F802BDC0460029F7D023
:401FC00076E7704703460B437FD4002243088B4274D303098B425FD3030A8B4244D3030B8B4228D3030C8B420DD3FF22090212BA030C8B4202D31212090265D0030B8B42EC
:4020000019D300E0090AC30B8B4201D3CB03C01A5241830B8B4201D38B03C01A5241430B8B4201D34B03C01A5241030B8B4201D30B03C01A5241C30A8B4201D3CB02C01A04
:402040005241830A8B4201D38B02C01A5241430A8B4201D34B02C01A5241030A8B4201D30B02C01A5241CDD2C3098B4201D3CB01C01A524183098B4201D38B01C01A52416A
:4020800043098B4201D34B01C01A524103098B4201D30B01C01A5241C3088B4201D3CB00C01A524183088B4201D38B00C01A524143088B4201D34B00C01A5241411A00D2BB
:4020C00001465241104670475DE0CA0F00D04942031000D34042534000229C4603098B422DD3030A8B4212D3FC22890112BA030A8B420CD3890192118B4208D389019211C2
:402100008B4204D389013AD0921100E08909C3098B4201D3CB01C01A524183098B4201D38B01C01A524143098B4201D34B01C01A524103098B4201D30B01C01A5241C308EF
:402140008B4201D3CB00C01A524183088B4201D38B00C01A5241D9D243088B4201D34B00C01A5241411A00D20146634652415B10104601D34042002B00D549427047634661
:402180005B1000D3404201B5002000F005F802BD0029F8D016E770477047C046002B15D1002A13D1002906DB01DC002806D00020C043410802E080210906002007B4024854
:4021C00001A14018029003BDD1FFFFFF03B4684601B5029800F04AF8019B9E4602B00CBC7047C046F0B54F464646C0B41604360C9946330005042C0C070C150C63437E43A3
:402200006F4365431C0CAD1964199C46A64203D980235B02984647446346250CEF191D044B464A4343432D0C240464199918C91920000CBC90469946F0BDC0469E2110B5DE
:40224000C905041C01F064FC002803D1201C00F053FD10BD9E21201CC90500F0C7FB00F04BFD80231B069C466044F2E7F0B583B016001F000090019101F072FC04000D0065
:4022800002000B0030003900FFF7ACFF009A019B121A8B41089920000A604B60290003B0F0BDC046F8B54A02430244004E00C50F240E28009B09360EC90F92098D4259D023
:4022C000A01B002800DC8DE0002E1AD1002A00D079E05A0704D00F221A40042A00D004335A0138D50134FF2C00D189E028009B015B0AE4B25B02E4055B0A2343C00718435D
:40230000F8BDFF2CE5D08021C9040A431B2800DD89E016002021C640081A8240511E8A4132439B1A5A0114D59B019E09300001F0F9FB05388640844265DC041B33002020E7
:402340000134E340041BA640721E964100243343BFE75A07BFD1DF082800FF2C2FD1002F00D187E08022D20313003B435B025B0AFF24BFE7A11B002949DD002E29D0FF2CD7
:40238000A7D08026F60432431B2900DD8DE017002026CF40711A8A40511E8A413A439B185A01D6D50134FF2C64D0012276491A405B080B4013438CE7031ECAD100207B0232
:4023C0005B0AE4B296E701380028AAD0FF2C9DD17FE7002A00D17CE701390029DFD0FF2CD2D176E7002820D1601CC0B2012853DD80279E1AFF0437402FD0D61A0D0095E73F
:402400002800002376E7614B241A334061E700294DD1611CCEB2012E2FDDFF292AD09B185B080C0055E701227BE7002C1BD1002B5BD0C04300280CD0FF2E7ED01B2800DDBB
:4024400092E01D002024C540201A8340581E83412B43D31A34000D0064E7002E00D065E700200024ABE7FF2E67D08024E40440422343E3E7FF2400233CE7002C61D1002BB2
:402480007ED0002A00D124E79B185A0100D460E73E4A0C0013401CE7002C1ED1002B2FD1002A66D013000D0013E7012277E7002C1FD1002B5AD0C94300290BD0FF2E50D0A6
:4024C0001B295FDC1F002024CF40611A8B40591E8B413B439B18340062E7002B1CD1002A4AD013000D00FF24F3E6130034000D00EFE6FF2E35D08024E40449422343DFE79E
:40250000002A00D1E5E68027981AFF04074000D152E7D31A0D00DCE6FF24002A00D1D8E68020DB08C003034204D0D208024201D113000D00DB00FF24CBE61300FF240D002F
:40254000C7E6002B0DD0FF24002A00D1C1E68021DB08C9030B42EDD0D2080A42EAD11300E8E71300FF24B4E6012372E713003400AFE60027002022E780270020FF03F1E6AB
:402580001300A6E60123A5E7FFFFFF7DFFFFFFFBF0B5564644465F464D46F0B444024600C70F83B08846650A360EBA463DD0FF2E22D00023EC00802599469B46ED042543A4
:4025C0007F3E43465C025800DB0F640A000E984636D0FF2830D080230021E400DB041C437F38301A0190484642460843724E800030587A4013008746002D44D108239946E7
:40260000063B9B46DDE70122FF2000241A406402C305640AD2071C431443200003B03CBC90469946A246AB46F0BD002D20D104239946033B9B46C4E7002C17D1022102E0BC
:40264000002C0AD10121321A01924A4643460A435A48920082587B409746200001F062FA431F76309C4040420021BAE70321B8E7280001F057FA431F9D40002376304642F4
:4026800099469B469DE70C239946093B9B4698E780240022E403FF20B9E70024C2468B465A465346022AAED0032A7DD0012A31D1012200201A400024A9E70122101A1B2850
:4026C00056DD1A4000200024A1E78023DB031D424BD18023DB032B435C02640A3A00FF2095E76D016001854230D2019A0024013A01921B220127290064006D00002901DB6C
:40270000A84201D82D1A3C43013A002AF3D16A1E95412C4301987F300028CEDD620704D00F222240042A00D00434220103D5244A019814408030FE2800DD64E70122A401DD
:40274000640AC0B21A4062E72C00A9E72D1A1A220124CFE76B02BCD500248023DB031C436402640A4246FF2051E71C42B3D1F4E721002022C140101A8440621E94410C4354
:40278000620704D00F222240042A00D00434620104D5012201201A40002438E70122A401640A1A40002032E78023DB031C436402640A5246FF202AE75C4A00009C4A000025
:4027C000FFFFFFF7F0B557464E4645464300E0B446028846760A1F0EC40F002F47D0FF2F25D0002380259A469946F600ED042E437F3F434642465D02D20F5B006D0A1B0EC5
:40280000904640D0FF2B39D080220020ED00D20415437F3BFB1842465746591C62408C4607430F2F5CD86F49BF00C9598F46002E45D108239A46063B9946DAE742460228BB
:402840002DD0032800D1C3E0012800D0A2E0002500260240D4B27602ED05760A2E43E407264330001CBC90469946A246F0BD002E1AD104239A46033B9946BAE72A00511EB6
:402880008A41901CC6E70120002DC3D0280001F049F9431F76309D4043420020BAE70124FF2514400026D6E7300001F03BF9431F9E400023763047429A46994699E70C23B8
:4028C0009A46093B994694E780260024F603FF25C1E735004846B2E7350022004846AEE72904090C0800370C3604360C2C0C7943704367437443060C64183619B14203D938
:4029000080214902884647440004000C310409188D01681E8541890E2943350CED19AD010D43290104D5012369081D4063460D4319007F31002925DD680704D00F2028400E
:40294000042800D00435280103D5274980330D401900FE29A3DC0124AD016E0A1440CDB279E78020C003064207D0054205D128434602760A4446FF256DE706437602760A5F
:40298000FF2568E70124611A1B2905DD14400025002660E76346CBE72E002023CE40591A8D406B1E9D412E43730704D00F233340042B00D00436730104D5012401251440EE
:4029C000002648E70124B601760A1440002542E780260124F6032E437602760A1440FF2539E7C046DC4A0000FFFFFFF7F8B54A024E0043024400240EC50F9B09360EC90F09
:402A00009209FF2E00D183E001204140A01BA9425CD0002800DC95E0002E1CD1002A00D081E05A0704D00F221A40042A00D004335A013BD50134FF2C00D191E001209B0178
:402A40005B0AE4B205405B02E4055B0AED0723432B431800F8BDFF2CE3D08021C9040A431B2800DD90E016002021C640081A8240511E8A4132439B1A5A0115D59B019E0980
:402A8000300001F04FF80538864084426CDC041B330020200134E340041BA640721E964100243343BDE70D005A07BCD1DF0801231D40FF2C33D1002F00D190E08022D20390
:402AC00013003B435B025B0AFF24BCE700284FDD002E2ED0FF2CA4D08025ED042A431B2800DD97E016002025C640281A8240501E824132439B185A01D5D50134FF2C6DD0A4
:402B000001227B481A405B08034013430D0088E7002A00D07AE777E7031EC5D100257B025B0AE4B28FE701380028A4D0FF2C97D177E7002A00D174E701380028DAD0FF2C08
:402B4000CDD16EE7002821D1601CC0B2012858DD80279E1AFF0437402FD0D61A0D008FE701231D4000236EE7624B241A334058E7002851D1601CC6B2012E33DDFF282DD07A
:402B80009B185B0804004CE7012274E7002C1AD0FF2E1FD08024E404404223431B2800DD96E01D002024C540201A8340581E83412B43D31A34000D005EE7002E00D05FE74C
:402BC00000250024ABE7002B44D0C0430028F0D0FF2EE3D11300FF240D0022E70D00FF24002330E7002C5DD1002B7DD0002A00D117E79B185A0100D456E73E4A0400134070
:402C00000FE7002C1ED1002B2FD1002A65D013000D0006E701226DE7002C1FD1002B59D0C04300280BD0FF2E4FD01B285EDC1D002024C540201A8340581E83412B439B1878
:402C4000340058E7002B1CD1002A49D013000D00FF24E6E6130034000D00E2E6FF2E34D08024E40440422343DFE7002A00D1D8E68027981AFF04074000D14DE7D31A0D0095
:402C8000CFE6FF24002A00D1CBE68020DB08C003034204D0D208024201D113000D00DB00FF24BEE6002B10D0FF24002A00D1B8E68020DB08C003034203D0D208024200D16B
:402CC0001300DB000D00FF24ABE61300FF24A8E601236EE713003400A3E6002700251EE780270025FF03E9E613009AE60123A6E7FFFFFF7DFFFFFFFB4302590A4300C20FB8
:402D00001B0E00207E2B0EDD9D2B0DDC802000040143952B0BDC9620C31AD9400B005842002A00D118007047034BD018FBE7963B99400B00F3E7C046FFFFFF7F70B50028E5
:402D400030D0C317C5185D40C40F280000F0EAFE9E231B1A962B0DDC9622D21A95406A02520AD8B25202C005520AE40702432243100070BD992B19DC9922D21A9540124AE9
:402D80002A40690704D00F210D40042D00D00432510103D50C4B1A409F231B1A9201520AD8B2DFE7002400200022DBE705222E00121AB921D6402A00C91A8A40551EAA41D2
:402DC00035001543DBE7C046FFFFFFFBF8B556465F464D464446F0B40F00FD0FAA4609037C002E005F00450F490A7F0D2943C5001803BC46400A570F640DDB0F3843D200DE
:402E00009A4500D1AAE06646A61B002E00DCFFE06346002B39D10300134300D0D9E06B0709D00F232B40042B05D02B1DAB42AD416D4249191D000B0200D482E0CA4B013478
:402E40009C4200D1FEE00A005646C84BED081A405007640552020543120B640D002112030B0D1B056405120B1A436308C04CF60714401C43640064083443280021003CBCD3
:402E800090469946A246AB46F8BDB74B9C42C6D080231B041843382E00DDEBE01F2E00DD1EE120239B1B9C4603006746BB40984613004746F3403B436746BA40571EBA4139
:402EC00013430200F240EB1A9D42B6411D008A1A7642911B0B0231D54A02560A002E00D1B4E0300000F01EFE0300083B1F2B00DDB5E020222900D21AD1409E400A009D408B
:402F000032439C4200DDB1E01C1B631C1F2B00DDD5E0202114002800C91A8C40D8408D400443DA40681E854111002543002476E74146314300D134E2310045466B0700D0A6
:402F40006FE756464807ED08C9080543864B9C4235D00A036405120B640D7FE76346E31A9B46002B00DC8BE06746002F3CD07E4FBC4200D153E780273F0438435B46382BC4
:402F800000DCF7E00243501E82410020D2B253194218AB4289411D00494289180B02CDD5714B01349C4200D13DE101206F4A6B080A4028401843D507054351082FE72B00F9
:402FC0000B4300D1CBE180231B030B431A03120B44E7013E002E6DD1AE1AB5429B41091A5B42C91A350075E70700174300D116E701235B429C46E3445B46002B00D0E0E0C3
:40300000AA18AA429B4109185B4259181500C5E7002E75D1661C7605760D012E00DCF3E0AE1AB0464545BF410E1A7F42F61B370200D48FE0551BAA42B641411A76428E1B77
:403040009A464BE756460022002507E7280000F069FD20300300083B1F2B00DC49E72A002838824000259C4200DC4DE73F49E41A1140D4E60243501E8241D3B2002222E7ED
:40308000002B00D0F3E0631C9C465B055B0D012B00DC9FE0344B9C4500D1C3E0AA180918AA42804140424118CD075208154349086446B4E62C4B9C4200D0ECE6AFE611009B
:4030C0001F3CE1400C00202B00D17FE04021CB1A9A4015436A1E95410021254300242DE733000700203BDF403B00202E70D04027BE1BB0400243501E824113430022E2E6D3
:40310000002C4FD0184CA44500D1ABE08024240476422143382E00DDDFE01F2E00DD43E12027BC1BA1460C004F46BC40A0462C004746F4403C434F46BD406F1EBD41F14021
:403140002C43151BAA429241411A5242891A64469A46BFE641464546314300D0BEE6002600240025F2E6C046FF070000FFFF7FFFFFFF0F801F2B59DC2027FF1ABC460700F2
:4031800063469F405B46B9461700DF40B8464F4643461F4363469A40531E9A415B463A43D840F4E60C002C435CD0F643002E55D1551BAA42A441411A6442091B9A46644630
:4031C00088E6964FBC4200D0D8E628E6002280E700208FE70B002B43002C00D0C2E0002B00D101E10300134300D118E6AB18AB42B6410918764271180A0200D409E1884A01
:403200001D00114064460AE6002C5BD10E002E4300D08AE00100114300D1C2E0010015009A46FCE56446002100258FE620235B429C46DC4463460700DF405B46BC46202BD2
:4032400000D1ACE040235F46DB1B98400243501E8241634613431A00002098E66F4CA44500D057E70100150064469A46D7E5002C39D10C002C436ED0DB43002B1AD0674C0B
:40328000A44568D0382B00DDA4E01F2B00DDAEE020240F00E41AA740B9462F00DF40B846A3464F46444627435C46A5406C1EA541D9403D43AD1895429B4109185B42591848
:4032C00064466BE60C002C4315D1010011437BD0010015009A46514CA1E50D43691E8D410021ECB22DE74D4CA44534D0802424045B422143C6E7040014434ED0ED084C0780
:403300002C438025C9082D03294208D0C6082E4205D1D208410711430C009A463100620FC900E50011433D4C79E50600164300D175E5AE1AB0464545BF410E1A7F42F61B68
:40334000370200D4F4E5551BAA42B641411A7642891B9A4663E50100150064465FE5002200257BE5002B3BD00300134315D0ED084B072B438025C9082D03294207D0C408AD
:403380002C4204D141070B002100D2081343C9005A0F1143DD00214C41E5204C3FE5002054E700260025D1E534000F00203CE7403C00202E2BD04027BE1BB1400D43691EF1
:4033C0008D4100212C43BCE6802100260903134C0025BBE50D43691E8D410021EDB269E7010015000D4C1AE50100150017E51C000F00203CE7403C00202B0CD04027FB1A14
:4034000099400D43691E8D410021254352E70021D4E71D0092E50021F3E7C046FF070000FFFF7FFFF0B55F4656464D464446F0B40D0399464E002B0B87B007009246804663
:403440009B46760DCC0F002E69D06D4B9E4235D05B468022DD001204430F13432B439B46C3009846674B00279C460023664401934A4615035000D20F53462D0B400D914651
:4034800000D176E05E4A90426CD080225B0F120413435C4AED0094461D4353460022DB00604449463618701C6140029017430F2F00D9AFE05448BF00C759BF465B461F4391
:4034C00000D088E000239B469846023308270193CEE74946022A6AD0032A00D109E2012A00D0BBE111400022002300259046CCB200212D030A0D12052D0B1543434A1B05C5
:4035000015401D436D00E4076D0825434046290007B03CBC90469946A246AB46F0BD034352D05B46002B00D18AE1584600F0FAFA03000B3B1C2B00DD7BE11D22D31A3A00E7
:4035400001005D46DA4008398D4013008F402B439B46B8462E4B00279C46002360444642019385E752462A432CD100250023022297E752462A4321D0002D00D154E1280042
:4035800000F0D0FA03000B3B1C2B00DD46E11D21CB1A51460200D9405346083A954093400D431B4A944660444042002279E7012400220C40124B0025904699E7002500237B
:4035C00001226EE703226CE700239B4698460133042701934CE703230C27019348E700238025984600242D03054B81E75D464346019A6FE75D4643462100019A6AE7C046A9
:40360000FF07000001FCFFFF1C4B0000FFFF0F80F30300004246120C91461A0C9446424617044A461B041B0C5A43604690464A4642431000039262461C003F0C7A437C434B
:4036400042440192220C9246019A5244904506D98246802040028046C24450460390100C049048462404240C1204121905922A0C2D042D0C68432C00824648467C4350431A
:403680008146200C8046574357444744BA4503D9802040028046C144380C3F04B84648442404240C01900498A044404404905846000C814658460404200C824607004846D7
:4036C0005F434C464343604660436446834650464443380C8446E4186444A34203D980235B029C46E34448463F04230C3F0C2404E419574668436F4384464D4650465543C6
:403700004243380C814662444A445B44944503D9802040028446654403983F04834604983F0C8446E344C345804140428246100484460198674484466744A344BC46A34522
:40374000A4419946D44464428742BF41D4458041E144A04699459B417F424042C8440743120CBA18A045A4415F423B0064422343D71843467D19DB0D6D021D435B465A0262
:40378000059B1A43531E9A415B46DB0D1A4343465B021343EA0107D501225C0813402343EA07029E13436D08574AB218002A4BDD580709D00F201840042805D0181D9842AF
:4037C0009B415B42ED180300E80104D54F4A15408022D200B2184E48824200DDE7E60124DB08680718436D02530580462D0B5B0D0C407DE6802259461203114208D01542D0
:4038000006D115432D0398462D0B4C46414B6FE65D4615432D032D0B3E4B69E603005546283B9D400023BCE6504600F07BF92030A8E60300283B9F400023BB46984689E634
:4038400000F070F9203073E60124A61A382E07DD00220C4000230025904649E6029EA3E71F2E20DC20222C001800921BF040944093400443581E83411C43F540630709D087
:403880000F232340042B05D023001C1D9C4292415242AD182B021FD5012400220C4001230025904624E61F202C004042821AD440202E1CD04022961BB5402B43581E8341A5
:4038C0000720234318400025002809D00F2200251A401C00042AD8D1230068076D022D0B0124DB08034398460C40002300E60025E3E780220124120315432D0398462D0BF7
:403900000C40044BF4E5C046FF030000FFFFFFFEFE070000FF0700000B0330B5134D1A0B4B005B0DC90F0024AB4211DD104CA34210DC8024640322430E4CE41A1F2C0CDDDA
:403940000D48C31ADA4013005C42002900D11C00200030BD094BCC18FAE7E040084CA44663449A4013000343EEE7C046FE0300001D0400003304000013040000FFFFFF7F0F
:40398000EDFBFFFF70B5002830D0C317C4185C40C50F200000F0C6F8174B184A1B1AD21A1F2A18DD164AD21A9440002224035B05240B5B0D0021100024030A0D1205240BA8
:4039C0001443104A1B0514401C436400ED0764082C43210070BD210091400A000B21081AC4405B052403240B5B0DE3E70025002300240022DEE7C0461E04000033040000DA
:403A000013040000FFFF0F804200120E511C4302C9B270B55D0AC40F012915DDE02189008C466D071B0B6244002128000D0D2D052B431C4D52052B40520813435B00E40718
:403A40005B082343190070BD002A15D1002D1FD0280000F067F80A281DDC0B232A001B1ADA4013000200153295400F4A1B03121A52051B0B520DD7E7002D06D080221B0B89
:403A8000120313436D07094ACEE7084A0023CBE700220023C8E703000B3B9D402B000025E3E7C046FFFF0F8089030000FF0700008446081C6146FFE71FB500F09BF90028A4
:403AC00001D40021C8421FBD10B500F027F94042013010BD10B500F08DF9002801DB002010BD012010BDC04610B500F083F9002801DD002010BD012010BDC04610B500F0A8
:403B000035F9002801DC002010BD012010BDC04610B500F02BF9002801DA002010BD012010BDC0461C2101231B04984201D3000C10391B0A984201D3000A08391B09984215
:403B400001D30009043902A2105C40187047C04604030202010101010000000000000000F0B544465F4656464D46F0B41C0083B0002900DA92E00F00002106008A46100076
:403B80001900002C00DA80E034003D0081468846B94269D866D04146484600F06FF983463900300000F06AF95B461B1A9C46203B9B4600D586E04946584681400B00494665
:403BC000604681400A00BB4200D971E06DD034003D005946A41A9D41002900DA89E00021002001260090019159468E400196614601268E4061460096002960D0D9075608DA
:403C00000E435F086146012200230CE0AF4201D1A6420AD8A41BBD4124196D410139A4185D41002906D0AF42F0D9013924196D410029F8D15B460098019900196941002B99
:403C40004CDB2E00DE4063462C00DC405B46002B5ADB34009C4023006446A6403200801A994103E0B04296D9002000215346002B04D003000C0000215842A14103B03CBC02
:403C800090469946A246AB46F0BD5346DB430C009A46130000215842A14175E7002746428F41012149428A4669E7B14200D88EE70021002000900191614600299ED1009854
:403CC0000199D3E7624640462023494690409B1AD9400300009100990B4370E7624620239B1A2A009A40260013006246D6401E43A9E7614620260127761A00200021F74057
:403D000000900191019772E762462023350094409B1ADD4023002B439EE7C046430270B542004C005D0AC30F4802120E460A240EC90FFF2A0FD0FF2C11D00120A24200D0B0
:403D400070BDB542FCD18B420DD0002AF8D12800431E9841F4E70120002DF1D1EBE70120002EEDD1E9E70020EAE7C0464302F0B542005D0AC30F4802440A4800120E000E4F
:403D8000C90FFF2A1FD0FF2822D0002A09D16E426E4100280FD1002C0DD10020002D09D005E0002801D1002C01D08B4213D0584201231843F0BD002EF7D0484241410120EB
:403DC00049420843F6E7002DDDD002204042F1E7002CDAD0F9E78242E9DC04DBA542E6D80020A542E6D25842434101205B421843E0E7C0464302F0B542004C005E0AC30F82
:403E00004802120E450A240EC90FFF2A17D0FF2C19D0002A0BD170427041002C17D0002807D048424141012049420843F0BD002C13D08B4214D0584201231843F6E7022098
:403E4000002EF3D1E3E70220002DEFD1E1E7002DE5D10020002EE9D0EDE7002DE9D1EAE7A242E8DC04DBAE42E5D80020AE42DDD25842434101205B421843D7E710B5002963
:403E800003D1FFF74FFE203002E0081CFFF74AFE10BDC046014B18687047C046780100200E4B70B500251E000D4CE41AA410A54204D0AB00F35898470135F8E700F06AFE99
:403EC000084B00251E00084CE41AA410A54204D0AB00F35898470135F8E770BDA04B0000A04B0000A04B0000A84B0000002310B59A4203D0CC5CC4540133F9E710BD0300E5
:403F00008218934202D019700133FAE7704700000EB410B59DB002A9029008610B48822488604861012040421FABC881084804CBA400006801938C8100F06EF80023029A50
:403F400013701DB010BC08BC03B01847FFFFFF7F78010020F0B58E6885B007000C00039201939E4243D890238A89DB001A423ED003250969236801985B1A029363695D43F4
:403F8000EB0F5D19029B6D1001331B18AB4200D91D00530510D52900380000F037FB061E14D0029A2169FFF7A1FFA289194B134080221343A38112E02A00380000F086FBE6
:403FC000061E0CD12169380000F0D4FA0C23402201203B60A38940421343A38117E0029B2661F61826606561019EED1AA560019BB34200D21E0032000399206800F0A5FA45
:404000000020A3689B1BA36023689E19266005B0F0BDC0467FFBFFFFF0B59FB0029005938B890F0016001B0610D50B69002B0DD1402100F0EBFA38603861002804D10C2387
:40404000029A01381360D8E040237B61002306AD6B6120336B761033AB7634002378002B03D1A31B049312D003E0252BF9D00134F4E7A31B320039000298FFF76BFF431C34
:4040800000D1B4E06A69049B944663446B612378002B00D1ABE00122002352426A6002A95432521801342B60EB60AB601370AB65534E21780522300000F03CFA002807D01C
:4040C0000123801B83402A68013413432B60EFE72B68DA0604D55322202102A8121811701A0704D553222B2102A81218117022782A2A03D0099B00200A210EE0059A111DEE
:4041000012680591002A01DB099204E05242EA60022213432B6001340BE02278303A092A04D84B4301349B180120F6E7002800D0099323782E2B1ED163782A2B0AD1059B3E
:4041400002341A1D1B680592002B01DA01235B42079310E000230A201A0001346B6021783039092904D84243013452180123F6E7002B00D00792234E21780322300000F0E8
:40418000D9F9002806D04023801B83402A68013413432B60217806221B48661C297600F0C9F9002812D0194B002B06D10722059B073393430833059314E005AB00933A0042
:4041C000134B2900029800E000BF07E005AB00933A000F4B2900029800F08AF80390039B013304D06B69039A9B186B6135E7BB890B985B0601D5012040421FB0F0BDC04684
:404200005E4B0000644B0000684B000000000000553F0000F7B5170001938A680B6900900C00934200DA130022003B6043321278002A01D001333B6023689B0602D53B6898
:4042400002333B60062523681D401ED0230043331B785A1E9341226892061CD53020E1184331087021005A1C45310978A2184332023311700FE02200012319320199009888
:40428000089EB047431C0ED00135E3683A689B1A9D42F0DBDAE72200019943320098089DA847431C02D10120404220E006232068E1683A6803400025042B03D18D1AEB43D3
:4042C000DB171D40A3682269934201DD9B1AED180027BD420AD0220001231A3201990098089EB047431CDED00137F2E70020FEBDF0B58BB006920A00433207930590049256
:404300000A7E0C00109B6E2A00D1ABE011D8632A22D009D8002A00D1B5E0582A00D0C5E045310A70814A4FE0642A1DD0692A1BD0BCE0732A00D1AAE009D86F2A29D0702AF6
:4043400000D0B3E0202209680A43226037E0752A1FD0782A33D0A9E00E001A684236111D196013683370A4E021681A68080606D4490604D5111D19600023D55E02E0111D0C
:4043800019601568002D3BDA2D23049A6D42137036E021681A68080606D4490604D51568111D1960ADB202E0111D196015685F4B227E039308276F2A1DD00A271BE0220008
:4043C0007821453211705A4A19680392081D226818600D68100602D4500600D5ADB2D30702D520231A4322601027002D03D1202322689A4322602300002243331A7002E002
:404400000A274A4B03936368A360002B09DB0422216891432160002D05D1049E002B11D07BE0002D79D0049E28003900FDF7C6FD039B013E5B5C280033703900FDF738FD42
:40444000051EF1D1082F09D12368DB0706D563682269934202DC3023013E3370049B9B1B23612BE009681A68080607D4490605D5111D19601368A28A1A8004E0111D196064
:40448000136862691A600023049E236116E01A68111D1960166800216268300000F04AF8002801D0801B6060636803E0260042363270012323610023049A1370079B09AA86
:4044C00000932100069B0598FFF7A4FE431C02D10120404227E02369320006990598079DA847431CF4D0236800259B070FD4099BE068984217DA180015E02200012319321C
:4045000006990598079EB047431CE1D00135E368099A9B1A9D42F0DBE9E72600039B42361B7833708EE70BB0F0BDC0466F4B0000804B0000C9B28218904204D003788B4263
:4045400002D00130F8E70020704710B5884202D98B18984201D3002305E09B1A013A08D3995C8154FAE7934203D0CC5CC4540133F9E710BD70B50500002944D00C1F236863
:40458000002B00DAE418280000F0D8F81E4A13681100002B02D16360146031E0A3420DD92268A018834203D118685B688218226063600C6024E0A24203D813005A68002AE2
:4045C000F9D11E689819A0420BD12168711858181960824214D110685268411819605A600EE0A04202D90C232B6009E021686018824203D1106852684118216062605C6029
:40460000280000F09CF870BDF0010020032370B5CD1C9D43083506000C2D01D20C2501E0002D01DBA94202D90C23336048E0300000F084F8234B1C681A002100002913D08D
:404640000B685B1B0DD40B2B02D90B60CC181EE08C4202D1636813601AE04B6863600C0016E00C004968E9E7174C2368002B03D1300000F051F820602900300000F04CF8D1
:40468000431C18D00323C41C9C43A0420DD12560300000F054F8200007220B30231D9043C31A0ED05A42E2500BE0211A300000F033F8431CEBD10C233000336000F03FF858
:4046C000002070BDF0010020EC010020F8B506000C001500002904D11100FFF797FF040018E0002A03D1FFF745FF2C0012E000F027F885420ED929003000FFF787FF071ED7
:4047000007D021002A00FFF7F1FB21003000FFF731FF3C002000F8BD002370B5064C050008002360FCF726FC431C03D12368002B00D02B6070BDC046900500207047704714
:404740000B1F1A68101F002A04DA891804390B68D0180438704700000000000004F4FF7F010000003432306D413A0000517569636B496F542D34746F32306D410D0A0000C1
:404780005061636B657420696E6974004144432070726F636573732073746172740D0A0054696D65722073746172740D0A0000004D6F64627573207374617274200D0A002C
:4047C0002025640000000000000000000000000000000000000000000000000000000000000000000000000000000000000000000000000000000000000000000000000010
:40480000000000000000000000C1814001C0804101C0804100C1814001C0804100C1814000C1814001C0804101C0804100C1814000C1814001C0804100C1814001C080415C
:4048400001C0804100C1814001C0804100C1814000C1814001C0804100C1814001C0804101C0804100C1814000C1814001C0804101C0804100C1814001C0804100C1814018
:4048800000C1814001C0804101C0804100C1814000C1814001C0804100C1814001C0804101C0804100C1814000C1814001C0804101C0804100C1814001C0804100C18140D8
:4048C00000C1814001C0804100C1814001C0804101C0804100C1814001C0804100C1814000C1814001C0804101C0804100C1814000C1814001C0804100C1814001C0804198
:4049000001C0804100C1814000C0C101C30302C2C60607C705C5C404CC0C0DCD0FCFCE0E0ACACB0BC90908C8D81819D91BDBDA1A1EDEDF1FDD1D1CDC14D4D515D71716D61F
:40494000D21213D311D1D010F03031F133F3F23236F6F737F53534F43CFCFD3DFF3F3EFEFA3A3BFB39F9F83828E8E929EB2B2AEAEE2E2FEF2DEDEC2CE42425E527E7E626D7
:4049800022E2E323E12120E0A06061A163A3A26266A6A767A56564A46CACAD6DAF6F6EAEAA6A6BAB69A9A86878B8B979BB7B7ABABE7E7FBF7DBDBC7CB47475B577B7B67697
:4049C00072B2B373B17170B0509091519353529296565797559594549C5C5D9D5F9F9E5E5A9A9B5B99595898884849894B8B8A4A4E8E8F4F8D4D4C8C448485458747468657
:404A0000824243834181804000300F40000400400F4000046F08DA80222086208708A708C810000002400F4005410F40030405060708090A0B0C0E0F10111213141516175B
:404A400018191B1C1D1E1F2021222325262728292A2B2E2F3031323334350000E226000006260000C42600009C260000C426000090260000C42600009C26000006260000F2
:404A800006260000902600009C260000482700004827000048270000CA2600000626000006260000B02600009A260000B026000090260000B02600009A26000006260000D9
:404AC00006260000902600009A26000048270000482700004827000054270000E02800003E2800003E2800003C280000D2280000D2280000C82800003C280000D2280000D2
:404B0000C8280000D22800003C280000D8280000D8280000D82800006229000014360000D4340000D4340000D2340000EC350000EC350000DE350000D2340000EC350000C0
:404B4000DE350000EC350000D2340000F4350000F4350000F4350000F43700004300232D302B2000686C4C0065666745464700303132333435363738394142434445460081
:404B80003031323334353637383961626364656600000000F8B5C046F8BC08BC9E467047C5010000ED0F0000F8B5C046F8BC08BC9E4670479D010000104C0000C00000206B
:404BC000C0000000180400000000E803A6004803000000000000000000000000A600EA002D017101B401F7013B027E02C2020603480300000000000000000000000000004B
:404C00000000000000000000010000000000000000000000070014000A00E80332006400190000000202020204080E1A1A0034004E009C0039017102E204C40900010203DA
:404C400098050020000104400100000003000000010000000000E02EC05D00001800000000366E010404040000000000000000000000000000000000000000000000000039
:404C800000000000000000005C4B0000000000000000000000000000000000000000000000000000000000000000000000000000000000000000000000000000000000004D
:404CC000000000000000000018010020000000000000000000000000000000000000000000000000000000000000000000000000000000000000000000000000000000007B
:404D00000000000000000000000000000000000000000000000000000000000000000000000000000000000000000000000000000000000000000000000000000000000073
:404D40000000000000000000000000000000000000000000000000000000000000000000000000000000000000000000000000000000000000000000000000000000000033
:404D800000000000000000000000000000000000000000000000000000000000000000000000000000000000000000000000000000000000000000000000000000000000F3
:404DC00000000000000000000000000000000000000000000000000000000000000000000000000000000000000000000000000000000000000000000000000000000000B3
:0200000490303A
:020000005BDFC4
:0200000490402A
:200000000000000000000000000000000000000000000000000000000000000000000000E0
:0200000490501A
:0C000000000204C81193110104E16D72AC
:0200000490600A
:0100000001FE
:00000001FF